:030000000219FDE5
:03000B000200AA46
:03002B0002015D72
:03005B000202EFAF
:030073000202DCAA
:1000800002030406080C10182030406080040608A3
:100090000C10182030406080A0C00003070F1F0D17
:1000A0000D0403060D0503030202C2AFC0D0C0E079
:1000B000206214E5256009E473E525F4F58AD2622F
:1000C000D0E0D0D0D2AF3285268AC262E526F46075
:1000D0003030682620720DD0E0D0D0C290C291C2DC
:1000E00092D2AF32C290C291C292206F0D20650AA7
:1000F0007401D5E0FDE57BF45290D0E0D0D0D2AFD2
:1001000032758A00C28DD26201FA01B930680520C9
:100110006502D29001B9306805206502D29101B91B
:10012000306805206502D29201B9D29330680A2066
:1001300065077405D5E0FDD29001B9D29430680A04
:100140002065077405D5E0FDD29101B9D2953068DC
:100150000A2065077405D5E0FDD29201B9C2AFC28D
:10016000AD53E6EFC0D0C0E0D2D3D2AFC2CEE52AC5
:10017000600720744F152A21C47800790020742E5E
:10018000E580307E01F430E60278FF53DACF207E3E
:100190000343DA20307E0343DA10C2D8C271E5800F
:1001A000307E01F430E60279FFC3E89970CB30610C
:1001B00003752A40207403752A40885CD270E86079
:1001C00003755F0020740DE52B6004152B21D443CB
:1001D000DA01C2D820700221E7A85C206102C27057
:1001E00020740221E588227882B604038522242027
:1001F000CF0AD0E0D0D043E610D2AD32C2CF053A1C
:100200007802E52A6005307402152AC3E55C940182
:100210004005755F004128756000756900E55F2441
:1002200001F55F5003755FFF7982B7020D306E1DD7
:10023000C3E52294324016854C227982B7030E30F2
:100240006E0BC3E52294324004798E8722C3E523E6
:100250009522600840041523415C0523D8CA05692E
:10026000E56970021569D56A69756A017808E56BF8
:1002700060497805C3E569956B4057C3E569956C9E
:1002800050087801756A03020296C3E569956D50BE
:10029000057801756A01C3E5629524401E7982B72D
:1002A000040241C7206E14852462E5690460038559
:1002B0006B69756A0175233C0202D2E5622850051C
:1002C0007562FF41C7F562E5620470067560FF75EF
:1002D00069FFD0E0D0D043E610D2AD32C2AF53E6D2
:1002E0007F7592FA7593FFC260759104D2AF32C2E6
:1002F000AF53E6EFC2ADC0D0C0E0C0F0D2D3D2AFB2
:10030000A8FBA9FCC2D8307102615653DACF207E17
:100310000343DA10307E0343DA20D271E580307E69
:1003200001F420E602612D88278928A13B53DACF0A
:10033000207E0343DA20307E0343DA10C2D8C27134
:10034000307402A1277800E580307E01F430E602A7
:10035000A127885CA10F53DACF207E0343DA203037
:100360007E0343DA10C271206102812F53DACF205D
:100370007E0343DA10307E0343DA20C2D8D271887C
:10038000578958C3E89555F8E99556F97B007E08DA
:100390007A00C3E8948CE994005005755B008121D4
:1003A000882178A2E6A8216055C3E894C8E99400A2
:1003B0005008E4D2E4FB7A0A61FCC3E89468E9944B
:1003C000015008E4D2E3FB7A0F61FCC3E894D0E962
:1003D00094025008E4D2E2FB7A1E61FCC3E894A0C8
:1003E000E994055008E4D2E1FB7A3C61FCC3E8944F
:1003F00098E994085008E4D2E0FB7A787E00C3E8DC
:100400009559FCE9955AFD30E70AECF42401FCED1E
:10041000F43400FD755B00C3EC9AED9E5003755BF0
:10042000018859895A8557558558567802A10FC3B6
:10043000E89527F8E99528F9307C0281F3307B02B2
:1004400081F3307A0281EC2075028152E9FDE8FCEB
:100450008171E9C313F9E813F830790281ECE9C33B
:1004600013F9E813F830780281ECE9C313FDE813BF
:0F047000FC20612CC3EC941CED940240028188A7
:10047F00ED701EC3EC94C850180529E529700215BC
:10048F0029C3E529940A5002A127755C00D270A1F7
:10049F0027E529600215297400207F037896E6244A
:1004AF00FAFEE43400FFC3EC9EFCED9FFD5006788E
:1004BF0000790081F3C3EC94FFED9400400678FFC0
:1004CF00790081F3EC8572F0A4C5F0A2F733F879C7
:1004DF0000400302050F78FF790002050FE9C313EF
:1004EF00F9E813F8307C0EE9600278FFC3E813389F
:1004FF00F8E43400F9C3E894FFE99400400278FF70
:10050F00885CD270206102A127741FF4552F4BF520
:10051F002FC274EB7002D274752A40307403752A9F
:10052F000A306102A13B20740353DAFE2074037575
:10053F002B20D0F0D0E0D0D0D2AD43E610327901ED
:10054F0002056B790302056B790A02056B791E02AE
:10055F00056B796402056B79C802056B7817E4D5D2
:10056F00E0FDD8FAD9F6227A147B780205927A1038
:10057F007B8C0205927A0D7BB40205927A0B7BC8B5
:10058F00020592E573D5E001227902E4D294D5E019
:10059F00FDD291D5E0FDC291D5E0FDC294D5E0FD2D
:1005AF00E920E002D29030E002D292E573D5E0FD6F
:1005BF00E920E002C29030E002C2927496D5E0FDCD
:1005CF00D9C9EAF8D5E0FDD8FBDBB8D29422C37CB9
:1005DF00007D0075F00005F0EA33FAEB33FB50F6BF
:1005EF00EB13FBEA13FAC3E9FFE8FEE89AF8E99B7D
:1005FF00F95004EFF9EEF8B3EC33FCED33FDD5F021
:10060F00DFEDF9ECF822E889F08A20D2D4F8A9F0CE
:10061F007B0030F70B7BFFF42401F8E9F43400F989
:10062F00E88520F0A4ADF0F8E98520F0A4AFF0FE46
:10063F00ED2EF974003FFA7C04C3EA13FAE913F9BB
:10064F00E813F8DCF48BF030F70AE8F42401F8E94A
:10065F00F43400F9E889F0C2D4F8A9F0227882B610
:10066F00040302070BC3E55C9419401EE52D5406E5
:10067F007018206E3678057994E7146007780A149D
:10068F0060027812C3E54198401F306E098564629D
:10069F007569FF756A01852224E4F544F545F54631
:1006AF00F547F548C26E02070BD26E7994E71470C6
:1006BF0013E523F43333F913F8E9540104F9E8543B
:1006CF00FE0206FFE714147014E523F4333333F9F5
:1006DF0013F8E9540304F9E854FC020707E523F47F
:1006EF0033333333F913F8E954070404F9E854F8B2
:1006FF00C39440F8E99400F98844894522C3E54141
:10070F0013F9E54013F8C3E54498F8E54599F95016
:10071F000CC3E89480E994FF4016020743C3E894A2
:10072F007FE994005003020743787F790002074363
:10073F00788079FF8849894A22E5492546F8E54AB4
:10074F003547F9854A20E4300701F43548FA30E798
:10075F0009C3EA94F04015020781C3EA940F5003CE
:10076F0002078178FF79FF7A0F02078178007900FD
:10077F007AF0C3E5249561500AC374019524500B98
:10078F0002079FE54A20E70E02079FE54A30E7067A
:10079F00884689478A482278A5E6FAC3E54933F89F
:1007AF00E54A33F9D115E930E70BC3E89480E994B2
:1007BF00FF4013E1D9C3E8947FE994005002E1D9D7
:1007CF00787F7900E1D9788079FFE820E715C3E5D4
:1007DF002398F84009C3E894014003020800780108
:1007EF00020800E8F424012523F8400302080078EA
:1007FF00FF884B2278A6E6FAA847A948120615E902
:10080F0030E70CC3E89401E994FF4016020835C3A2
:10081F00E894FFE99400500302083578FF7900024D
:10082F000835780179FFE920E715C3E54B98F840C3
:10083F0009C3E89401400302085C780102085CE8F0
:10084F00F42401254BF8400302085C78FF8824222A
:10085F0078FF20692879A1E76023E541601F74FFC5
:0F086F008541F0848539F0306A0375F005A4F8EF
:10087E00C5F0600278FFC3E895645002A8648863EF
:10088E0022C3E5409440E5419401E5635003140111
:10089E00A0046002F563227883E6F520120F23751B
:1008AE00E89012054D75E89030EDFDA8BDA9BE1279
:1008BE000FCA756E80756F02C3740213FD7480606B
:1008CE006613FC74802CFC74023DFDECFAEDFBC348
:1008DE00E89AE99B4014E56E2480F56EE56F3402CC
:1008EE00F56FEA2CFAEB3DFB80E5AE6EAF6FC3E51C
:1008FE006F13F9E56E13F8C3E913F9E813F87A03E9
:10090E00C3E913F9E813F8DAF7AA201A7009756E1D
:10091E0000756F000209351AEA6008EE28FEEF39FD
:10092E00FFDAF88E6E8F6F2275E890227883E6FFDD
:10093E0030EDF9A8BDA9BE0570C3E570940840520C
:10094E00757000E9FA79A0E76044EA7007E5716016
:10095E001B02096EC3E895716010E5715006600CBC
:10096E001402097A0460F902097AE571F571C394EB
:10097E00F6401B7561C0C394064013756180C39425
:10098E0006400B756140C39406400375610075BB4C
:10099E000E22EFC39401601F7480601BC3E894FFA6
:1009AE00E994035012C3E8956EE9956F5009E5611D
:1009BE00600C15610209CCE561F460020561A86165
:1009CE00C3E524985002A824C3E89562400AA862A1
:1009DE00E562F4600385626188258826E570B407B8
:1009EE000375BB1022743279A787F0A4C5F0A2F765
:1009FE0033F8C3E895614002A861882288248825CF
:100A0E0088268864227540007541F022C2AF75C8F1
:100A1E0020A8CCA9CDAA3A30CF010A75C824D2AFEE
:100A2E00AB3BAC3C883B893CC3E89BF8E99C206916
:100A3E0008F9306602612B4185AD3D8A3DF9EA9D8C
:100A4E00FA600678FF79FF416AAE3EAF3F8B3E8C6F
:100A5E003FA83BA93CC3E89EF8E99FF9C3E54113C3
:100A6E00FBE54013FAE82AF540E93BF541500675DF
:100A7E0040FF7541FF41D2AA40AB41AC40AD417E33
:100A8E00047F02C3EB9404400D1E1FC3EB94084079
:100A9E0005206A021E1FC3ED13FDEC13FCDEF7C327
:100AAE00EA9CFAEB9DFBEF6009C3E913F9E813F832
:100ABE00DFF7EA28FAEB39FB8A408B4150067BFFC1
:100ACE008B408B41C3EB94025002D2663069047F97
:100ADE000341FD7892E6FFC3E537948240110FC3C0
:100AEE00E53794A040010FC3EF940640027F057EC8
:100AFE0002E541C4540FF9E541C454F0F8E540C491
:100B0E00540F28F8C3E89EFAE99400FB4009C3EAA3
:100B1E009402EB940050047A02E4FB6177AA40AB96
:100B2E0041EBC4FEEAC4540F4EFCC3EA9CFAEB94AC
:100B3E0000FBC3E813C313F8EA28FAEB3400FB8A70
:100B4E00408B41C3EB94024002C2667802EBC4FEB6
:100B5E007B00EAC4540F4EFAC3EA98FA4005C394D8
:100B6E000250027A027892E6FF3060026177855178
:100B7E0092855293D26043E680C3E49AF8E49BF9DF
:100B8E003066028103E8FAE9FBD3E913FDE813FCB2
:100B9E0088518952C3EF94036038EF20E00DE82CA2
:100BAE00F8E93DF9ECFAEDFB020BCCE828F8E9394F
:100BBE00F9C3E82402F8E93400F97AFE7BFFC3EFAB
:100BCE009403400E8A538B54884D894E8C4F8D5012
:100BDE008137885389548A4D8B4E8C4F8D50306996
:100BEE00127553F07554FF754FF07550FF7551F037
:100BFE007552FF8137E8FAD3E813FC8851C3EF949E
:100C0E00036020EF20E007E82CF8ECFA8123E828B7
:100C1E002402F87AFEC3EF940340088A53884D8C61
:100C2E004F813788538A4D8C4FE568C33350026429
:100C3E006BF5683060028141753402D26043E68004
:100C4E00E52D54066034A840A941C3E913F9E81311
:100C5E00F8C3E913F9E813F8306904E92440F9C23E
:0E0C6E00AF53E67F759100C3E498F594E499C6
:100C7C00F595759104D26043E680D2AF22D26475AB
:100C8C004300752000306C03752040020CA8D26420
:100C9C00754300752040306C037520007801790194
:100CAC00206620E52D54066002C2647914E541C328
:100CBC0013700104F8C3941440027814306904785A
:100CCC001B791B206010E543600C306903D534049C
:100CDC00D26DA15391490543E59BF45440B52002D4
:100CEC00A13D30690908C3E89940011881CF2064FF
:100CFC000A08C3E899400281A881CFC264C2AF53ED
:100D0C00E67F7591003066127594007595F87591B3
:100D1C0004D26043E680D2AF81A8E5417EFFC333A5
:100D2C004005C3334001FEC3E49E759400F595A1C4
:100D3C001AC3E5339401500281A830640281A8D80B
:100D4C0002A15181CFC26DC2AF53E67F7591008570
:100D5C005394855495759104854D92854E93D2602C
:100D6C0043E680D2AFE52D54066008206A020533B5
:100D7C00020D8F306D0D206C0A20640715811581D2
:100D8C000216382278003064027801E53775F007D6
:100D9C00A4F9E5F028F5F0E9A2F013A2F113A2F200
:100DAC0013F537C394785003753778C3E537953806
:100DBC004008D265C290C291C292306002A1C68531
:100DCC004F92855093D26043E68022207D16C2AFAD
:100DDC00754202D294C293306202D292D2AF759F06
:100DEC0011020FC7C2AF754202D294C29530620293
:100DFC00D290D2AF759F11020FC7307243207D2065
:100E0C00C2AF75420390013B757B10C292D29530F4
:100E1C006204D291C124C294D2AF759F01020FC754
:100E2C00C2AF75420390013B757B10C290D29330D8
:100E3C006204D291C144C294D2AF759F21020FC7F4
:100E4C00207D17C2AF754203900116C29230620228
:100E5C00D291D2AF759F01020FC7C2AF75420390FA
:100E6C000116C290306202D291D2AF759F21020F4F
:100E7C00C7207D16C2AF754204D293C29530620270
:100E8C00D291D2AF759F21020FC7C2AF754204D267
:100E9C0095C293306202D291D2AF759F01020FC7F7
:100EAC00307243207D20C2AF75420590012A757BBC
:100EBC0008C291D294306204D290C1CAC293D2AF0C
:100ECC00759F11020FC7C2AF75420590014C757B1F
:100EDC0020C291D294306204D292C1EAC295D2AFB0
:100EEC00759F11020FC7207D17C2AF754205900187
:100EFC000CC291306202D290D2AF759F11020FC713
:100F0C00C2AF754205900120C2913062EBD292D2F1
:100F1C00AF759F11020FC7207D16C2AF754206D266
:100F2C0095C294306202D290D2AF759F01020FC766
:100F3C00C2AF754206D293C294306202D292D2AF43
:100F4C00759F21020FC7307244207D20C2AF7542BD
:100F5C000190014C757B20C290D293306204D292E6
:100F6C00E170C295D2AF759F21020FC7C2AF754217
:100F7C000190012A757B08C292D295306205D290FD
:100F8C00020F91C293D2AF759F01020FC7207D173C
:100F9C00C2AF754201900120C290306202D292D24F
:100FAC00AF759F21020FC7C2AF75420190010CC2F1
:100FBC0092306202D290D2AF759F01C2652290012D
:100FCC000A757B00C290C291C292D293D294D295F0
:100FDC00C2622278807607087607087601087604C4
:100FEC000876FF0876FF08760B087602087601086B
:100FFC007601788C76010876000876B40876FF08BE
:10100C0076FF0876FF0876030876FF0876010876E7
:10101C00FF0876250876D00876780876C808760416
:10102C000876FF08760108760008767A08760708B5
:10103C0076010876010876000876FF08760022789B
:10104C0087E6FFC272BF0302D2727888C27DE63097
:10105C00E102D27DC27E7889E630E102D27EC3EF16
:0F106C0094026008758E01D27302107D758E009C
:10107B00C273227880E6149000809378A5F678816D
:10108B00E6149000809378A6F67886E61490008D8F
:10109B009378A7F6789FE6F87005756B0001C4C3CB
:1010AB00E8941140027811E82828F56B256B256B25
:1010BB0028F56C256B2828F56D7886E6F539C394F1
:1010CB00025003753902789CE67538FFB40203753C
:1010DB0038A0B4030375388278A3E61490009A9372
:1010EB00F566120FCA22227896E6FA7897E6FB7815
:1010FB0088E6B40305C3EB940EFB307F047A007BC8
:10110B00FFC3EB9AFCC3948250027C82757200057C
:10111B0072EC8572F0A4C3E5F0947D40F222D27F8D
:10112B0011F212055C12055C7A007B007C10120533
:10113B0052E55C2AFA74003BFBDCF37C04C3EB1333
:10114B00FBEA13FADCF7FEC27F11F222757C007505
:10115B007D00E5EF20E6037520000520903FFFE5BD
:10116B0020146006901DFF1460009304600375EF5C
:10117B001453D9BF7581C043FF8012054D75EF0421
:10118B0043B203E5B3240220E70DF521E5E320E0AC
:10119B00068521B343E301120FCA7580FF75A400C6
:1011AB0075F1D075D4BF75907875A53F75F2BF7585
:1011BB00D54075A60175E241120FCAE4F8F6D8FDC9
:1011CB00756801120FDF12168F78988673753001D0
:1011DB00C2AF12056612057612055C12057D12056B
:1011EB005C12058412055C1217C2120566120566A5
:1011FB00120561C2AF757C00757D0078FA79FA3003
:10120B008607D9FBD8F7021C00114B117E11F11187
:10121B00F278988673120FCA75881075890275C893
:10122B002475910475D84075A82275B80275E6909F
:10123B00759B80759D0075D10775BC5875BB0E7578
:10124B00BA1175E88012054DD2AF1208A57536009C
:10125B0053DACF207E0343DA20307E0343DA104388
:10126B00DA01C2D8C271120566D2617B037A0CE532
:10127B005B70077A0CDB030211FE12055C20700316
:10128B000211FEC270E55CC3940240E1E52F541FCE
:10129B00855E5DF55EB55DD5DAD5C26153DACF20DB
:1012AB007E0343DA20307E0343DA10C2D8C2717852
:1012BB00A2E67008D274E52F54E0F52FC27575299C
:1012CB0000120561307409C3E529940A4002D275F6
:1012DB0012055278023074027800C3E55C9840F036
:1012EB00C2AF120576120576120576D2AF120566DD
:1012FB00754C00120552788CE6C39401500302130F
:10130B00EBE530C3940150030213EB757CA5757D9F
:10131B00F1207435C3E55C94FF50030213EBC2AFAD
:10132B0012058BD2AF120561C3E55C940150EFC27D
:10133B00AF120576120557120576D2AF120561C3AF
:10134B00E55C94FF40E90218477F05D27F11F2124A
:10135B000561C2AFC27F11F2AE5CC3E55C947FD274
:10136B00AF500261FB12054DC2AF12058BD2AFDF3E
:10137B00DA3129C3EE94057897F61205661217CA6F
:10138B007F0AD27F11F2120561C2AFC27F11F2AE9A
:10139B005CC3E55C947FD2AF50E612054DC2AF1231
:1013AB000576120557120576D2AFDFD63129EE241A
:1013BB00037896F6F87997E7C39482400398500622
:1013CB00E824827897F61205661216DD1217F912C9
:1013DB00056111F2C3E55C94FF50026116021847D8
:1013EB00757C00757D00C3E55C954C4003855C4CBA
:1013FB0012056178017988E7B403027805C3E55CCF
:10140B0098400241FEC2AF12058B12058B12058B61
:10141B00D2AF120566753000E4F531F5320531E5D2
:10142B0031F4703F0532789AE678191460127832ED
:10143B0014600D787D14600878FA1460037532001F
:10144B00C3E53298401D120FCA12054D1532753186
:10145B000078998673C2AF12058BD2AF78988673DA
:0F146B00120561120557E52A700530740221FE43
:10147A0078012074027806C3E55C9840A1120561E0
:10148A00E52A70030211FEC2AF120FCAE4F522F573
:10149A0023F524F525F526F567D2AF7885E6C3331B
:1014AA00F565E4F544F545F546F547F548F570F573
:1014BA002CF52DF53775700875BB1012054D1209FC
:1014CA003630EDFDA8BDA9BEE97001F88871120990
:1014DA003A75700875BB10114BC2AF7561FF1209DE
:1014EA00F3852261852262852263D2AF7522017556
:1014FA002401752501752601856069756A01788858
:10150A00E6B40307C27D307602D27DD268D269750D
:10151A003300120F23120F52120A13120A1A120A56
:10152A0013120A1A120A13120C9A12066C120D904E
:10153A00120DD7120A1A120C89306E0312070C20E8
:10154A00660312085F30660312088F120D90120E9E
:10155A0006120A1A120C9A306E03120748120D90DC
:10156A00120E7D120A1A120C89306E031207A61285
:10157A000D90120EAC120A1A120C9A306E0312084F
:10158A0003120D90120F23120A1A120936120C892D
:10159A00120D90120F5212093A120A1A30692C854A
:1015AA006461856462856069756A0179187A0CC319
:1015BA00E533994009C269D26A8A350215D5C3E56D
:1015CA005C94014003021531021640306A25206CF2
:1015DA0022E535147006C26AD26BA131F535C3E52E
:1015EA005C940140030215317888E6C394036003D2
:1015FA00021640753600C3E55F94014009856462AE
:10160A00856069756A0178FA79A4E760027803C38C
:10161A00E55F985021307404E52A601A78F0306C3E
:10162A00058564617820C3E541985002A1310536E9
:10163A00E55C6002C143753600C2AF120FCA7887F3
:10164A00E6FE7602114B7887EEF6E4F522F523F5ED
:10165A0024F525F526F565752C00752D00D2AF12F7
:10166A000561120FCA78A4E66006D290D291D2928E
:10167A00307406E52A700221FE788DE6C394014093
:10168A000241DB8123901A0D782012171FE520B43E
:10169A00A50CA312171FE520B45A030216BD757CC8
:1016AA00A5757DF1120FDF1216DD757C00757D00C0
:1016BA000216DC901A0378807B0A12171FA308DB34
:1016CA00F9901A0F788C7B1912171FA308DBF9906F
:1016DA001A2822C2AF12176212173F901A00740E0C
:1016EA00121724A37409121724A37415121724902D
:1016FA001A0378807B0A121723A308DBF9901A0FC2
:10170A00788C7B19121723A308DBF91217751217A5
:10171A0053901A2822E493F622E6438F01538FFD51
:10172A00FFC3E583941C400122EF857CB7857DB712
:10173A00F0538FFE22438F02438F01857CB7857D4C
:10174A00B7901A0DF0538FFC22901A0D74A5F1244C
:10175A00901A0E745AF124227A3079D07820901A8D
:10176A0040F11FE520F709A3DAF7227A3079D09001
:10177A001A40E7F12409A3DAF922AB74A875BB0170
:10178A00027980BB02027981BB03027982BB04021F
:10179A007994BB05027983BB06027986BB07027975
:1017AA0092BB08027987BB0902799CBB0A02798835
:1017BA00BB0B027989E8F7227C05120566DCFB225D
:1017CA00C2AF12057612057D12058412058B120529
:1017DA005712057612057D12058412058B120557DC
:1017EA0012057612057D12058412058BD2AF22C22C
:1017FA00AF12058B12058412057D12057612055764
:10180A0012058B12058412057D12057612055712F0
:10181A00058B12058412057D120576D2AF22AE74AD
:10182A00AF75C2AF12057612057612057612055704
:10183A00DEF212058B120557DFF8D2AF221217CA51
:10184A001217C21217C275740175750175760011E7
:10185A00287C05AD5C120566C3ED955C70F5C3E5A1
:0F186A005C9401400AC3E55C94FF403702188A82
:101879001217841216DD1217CAC2AF75EF141217A8
:10188900C2DCD10576C3E5769403500280C21217F3
:10189900C20575E5741490009F93F808C3E575981F
:1018A900500280A91217C21217C20574C3E57494B5
:1018B9000C50028095120FDF1216DDC2AF75EF14BE
:0318C9001217C231
:0319FD000211577D
:101A00000E091507070104FFFF0B020101A55A018A
:101A100000B4FFFFFF03FF01FF25D078C804FF01DA
:091A200000FF07010100FF00FFB7
:101A40002353757065726D6963726F33703541230E
:101A500023424C48454C4923463333302320202031
:101A60002020202020202020202020202020202076
:101C0000C2AFC2D353D9BF7581C043B20343FF8073
:101C1000752438752503B1DC7529A5752AF175E29F
:101C20004043F14053A4BF75D4FFD2867DFA7803B8
:101C300079E67C10752200752300901DE97B0675FE
:101C400024987525013086028145208608D8FBD965
:101C5000F9DCF781B7308608D8FBD9F9DCF781B712
:101C6000B19CE493A3C39A6004DDC381B7DBDBB10D
:101C70008E6002812E7B08E493FAA3B16FDBF87AC1
:101C800030B16F752200752300B18EEAFCEBFDC305
:101C9000ED94FE400EB18E8A278B28ED30E0048A49
:101CA000828B83B18E7AC270D8C3ED94FE601950D6
:101CB000CEBD002BEC600F7520007521FF7529004B
:101CC000752A000200008100A827A9280809D80465
:101CD000D90281DCB192EA89AAF281CE0D81A3C337
:101CE000ED94035053EDA2E092007AC5C3E58294CF
:101CF00000E583941C508A200010438F02438F011B
:101D00008529B7852AB7F0300029A827A92808090E
:101D1000438F01538FFDD804D902A133C3E58394C7
:101D20001C4003A3A11689AAE28529B7852AB7F02A
:101D3000A3A116538FFC817F7AC1BD030CE493A34A
:101D4000FAB153DCF8B14B817F8181AA22AB23B178
:101D50006FEBFAEA6222752608C3E52313F523E543
:101D60002213F52250066323A0632201D526EAB18F
:101D7000DCB1DC75260AEAF4200102D286300102C9
:101D8000C286B1DCC3134002C201D526EB22B19258
:101D9000EAFB208602A192308602A197752608AE42
:101DA00024AF25C3EF13FFEE13FEB1E0B1DCC3EAAD
:101DB000133086024480FA30E703632201C3E5232F
:101DC00013F523E52213F52250066323A0632201B5
:101DD000D526D9E52265236523F52222AE24AF2539
:101DE0000E0FDEFEDFFCD20122424C48656C6934E6
:071DF000373164F3300601F6
:00000001FF
